:10000000C2C113C0189518951895189597C11895E1
:10001000189518950A600000B998C19A05B7026052
:1000200005BF0BB700640BBF08958A93FA93EA9358
:100030003A922A921A920A927A936A935A934A931C
:100040003A932A931A930A938FB7EAD08FBF0991F4
:100050001991299139914991599169917991099011
:10006000199029903990E991F9918991189543D186
:1000700050D1D2DF57D100E0E0E6008300E0E3E6B4
:10008000008300E213E0E1E60083118301E0E4E68F
:10009000008300E0E5E600830FEFE6E600830FEF64
:1000A000E7E6008300E0E8E6008300E0E9E600839D
:1000B00003E0E0E6008300E010E0E1E60083118366
:1000C00000E0E4E6008321D122D1FECFE6E6008104
:1000D0000F3F28F400916600039500936600E7E661
:1000E00000810F3F28F4009167000395009367009B
:1000F000E1E600811181012B39F0E1E600811181F7
:100100000150104000831183E0E60081015081F02E
:100110000A95B9F00A9579F10A9509F46DC0E1E6FE
:1001200000811181012B19F404E0E0E600830895B9
:10013000E1E600811181012B19F404E0E0E600837F
:100140000895E1E600811181012BA1F403E0E0E6CE
:10015000008304EF11E0E1E60083118301E0E9E6AA
:10016000008300E0E7E6008302E0E8E60083E9E6DA
:100170000081D2D00895E8E600810130E0F10091DD
:1001800068000A9500936800E8E60081002399F56D
:10019000E4E60081002349F1E9E60081002351F4FF
:1001A00001E0E9E6008300E0E7E6008301E0E8E63D
:1001B00000831EC000E0E9E60083E5E6008100233D
:1001C00021F4E6E600810A3260F0E1E60081118167
:1001D000012B39F400E0E5E6008300E0E4E600836B
:1001E00007C004E2E8E6008303C000E0E9E600831C
:1001F000E9E6008191D00895E8E60081013078F0C9
:10020000009168000A9500936800E8E600810023E9
:1002100031F400E0E9E60083E9E600817DD008954D
:10022000E6E600810B3008F465C0E0E6008101508D
:1002300099F00A9519F10A9529F10A9509F44BC02C
:1002400001E0E3E600830CE211E0E1E600831183C4
:1002500001E0E0E600834BC000916300039500934A
:100260006300E3E60081053040F00CE211E0E1E6D6
:100270000083118302E0E0E6008339C004E0E0E699
:10028000008335C0E1E600811181012B81F5E4E6B0
:100290000081002341F0E6E600810A3240F101E0EE
:1002A000E5E6008324C0E7E60081013200F1E6E6DE
:1002B0000081053218F401E0E4E6008301E0E9E69C
:1002C000008300E0E7E6008302E0E8E60083E9E679
:1002D000008122D00CC001E0E9E6008300E0E7E6FF
:1002E000008302E0E8E60083E9E6008115D000E043
:1002F000E6E6008308950CB701600CBF08B3056102
:1003000008BB05B7006205BF0895789408958895E5
:100310000895C39ABB9A0895002311F4C39A0895CF
:10032000C398089500E002BF00EA06BF02E00FBDD7
:1003300002E003BF09B7046009BF08958A93FA93E6
:10034000EA933A922A921A920A927A936A935A9369
:100350004A933A932A931A930A938FB7B7DE8FBFC3
:1003600009911991299139914991599169917991FD
:100370000990199029903990E991F99189911895EE
:1003800000008895FECF09E90DBFCAE806D000231A
:1003900009F00FD06CDEF4DFF3CF01E0089510E038
:1003A0001D930A95E9F7089515911D930A95E1F7B4
:1003B000089584E190E0FC010591A491FC0132963E
:1003C00025913491122F132B19F0F901EDDF01C0A3
:0E03D000E6DF049610E08831910768F3089587
:00000001FF
:00000001FF
